:020000040000FA
:040000001BEF00F002
:080008000A6AFA6AE836020FE9
:10001000F924F96E3F0C060C5B0C4F0C660C6D0C52
:100020007D0C070C7F0C6F0C770C7C0C390C5E0C74
:10003000790C710C120065EC00F0946A016A0150B1
:100040003DEC00F0FF0A63EC00F0320E45EC00F0EE
:1000500001503DEC00F0800FFF0A63EC00F0320E1F
:1000600045EC00F0012A01500908D8B039EF00F042
:10007000016A1FEF00F03BEF00F0026E02500F0B21
:1000800004EC00F0036E03501200026E0250036E87
:10009000640E046E010E4DEF00F0056EFF0E066E4D
:1000A0000450086E0350076EEF0E0624D8B055EFCB
:1000B00000F0072E54EF00F0082E52EF00F0052E4E
:0C00C00050EF00F012008B6E12001200D6
:0200000400F00A
:020000040030CA
:0E00000000260E0E00008000F0C00FE00F4042
:00000001FF
